:100000000C9426040C9443040C9443040C94430471
:100010000C9443040C9443040C9443040C94430444
:100020000C9443040C9443040C9443040C94430434
:100030000C9443040C9443040C9443040C94430424
:100040000C94F2070C9461050C9443040C94430443
:100050000C9443040C9443040C9443040C94430404
:100060000C9443040C9443040C9443040C944304F4
:100070000C9443040C9443040C9443040C944304E4
:100080000C9443040C9443040C944304281E0D2048
:100090002D1EF81F441E441E7E1E931EC51E141FD7
:1000A000901E0D200D20A91FBB1FD91FE71F0D207B
:1000B0000D200D200D200D200D200D200D200D20D8
:1000C0000D200D200D20FC1FFE1F032045617379BC
:1000D000436F6E74726F6C00204C4300696E636FE7
:1000E0006D70617469626C6520485700312E342E42
:1000F00033000102031304050611070809120A0060
:100100000B0C100F0E0D010101050D1F0C04040E48
:100110001F04041F0E040006091717090600000635
:1001200009121412090603070F1E1C1810000305FC
:100130000912141810000707070707070707070524
:100140000505050505071C101817150705071C10E0
:100150001817110202021C101812140605021C10B6
:100160001817140601061C101815150701011C109C
:100170001816110201061C101816110204071C1093
:10018000181216020207040A110A0A0E00000C17C0
:10019000141714170C001C101810160505051F0A5B
:1001A0000A0A0A0A1F000E11111F1B1B1F0002065C
:1001B0000F1F0F060200080C1E1F1E0C08000E0E5B
:1001C0000E0E1F0E0400040E1F0E0E0E0E00202039
:1001D000202020200000204D4D4920200000204DEF
:1001E0004D012020000020444343202000002053E4
:1001F000544F5020000053484F52542100002048D3
:10020000414C54200000000000000000000020507D
:10021000524F4720000052455345542000007E0EA7
:100220000E0E0E1B1B1C0E1B1B7E0E0E0E0E232D08
:10023000004144523A20256C6420202020202020B8
:10024000202020002D2D2D2D202000252D3564006F
:1002500025336400202001022020202020202000BF
:10026000252D356400252D31312E31317300414269
:10027000434445464748494A4B4C4D4E4F505152D6
:10028000535455565758595A30313233343536371E
:1002900038392E2C3A2D2B232F3D3C7C3E20004D0F
:1002A0004D20492020313420004D4D20492020325E
:1002B0003761004D4D20492020323762004D4D20DE
:1002C000012020313420004D4D20012020323761A3
:1002D000004D4D200120203237620044434320204E
:1002E0002031342000444343202020323820004471
:1002F0004343202031323820004C6F636D656E75AA
:1003000000000000000000000044434320686F6FBD
:10031000666473706F6F7200004C434420766572A0
:100320006C69636874696E67004C6F6B436F6E74C1
:10033000726F6C00000000000045786974000000D6
:100340000000000000000000004B69657A656E2027
:1003500000000000000000000044617461666F72DC
:100360006D61740000000000004E61616D2020206E
:10037000202020000000000000496E766F6572208A
:100380002020200000000000004D656E75204C6F9D
:10039000636F0000000000000050726F6772616DB3
:1003A0006D6174696F6E0000004C756D696E6F73DE
:1003B0006974650000000000004C6F6B436F6E7441
:1003C000726F6C0000000000004578697400000046
:1003D00000000000000000000053656C6563746954
:1003E0006F6E20000000000000466F726D61742087
:1003F000646F6E6E65657300004E6F6D2020202067
:10040000202020000000000000536169736965200E
:100410002020200000000000004C6F6B204D656E16
:10042000FC000000000000000044434320486175C8
:100430007074676C65697300004C43442042656CBE
:100440006575636874756E67004C6F6B436F6E748F
:10045000726F6C00000000000045786974000000B5
:1004600000000000000000000041757377E4686C34
:10047000656E20000000000000446174656E666FC8
:10048000726D617400000000004E616D65202020D7
:1004900020202000000000000045696E7472616732
:1004A0002020200000000000004C6F636F6D6F740F
:1004B000697665206D656E7500444343204D616922
:1004C0006E20547261636B00004C43442062616390
:1004D0006B6C696768740000004C6F6B436F6E74DF
:1004E000726F6C0000000000004578697400000025
:1004F00000000000000000000053656C656374207C
:100500000000000000000000004461746120666F7C
:10051000726D617400000000004E616D6520202046
:10052000202020000000000000456E747279202019
:10053000202020000000000000202D2D2D2D002562
:10054000357500536F6674772E205600312E342E89
:1005500033005365724E722E2025386C75003A2098
:100560000025357500253364002534643A20002DBC
:100570002D2D0025336400204F4B2020202000200B
:1005800020202020202000696E636F6D7061742E22
:1005900020466F726D617400496E636F6D702E201E
:1005A000466F726D6174202000466F726D61742019
:1005B000696E636F6D7061742E00696E6B6F6D7024
:1005C00061742E20466F726D6174002E2E2E20777E
:1005D000616974696E67202E2E2E2000233D6465AC
:1005E0006C657465000000000000000000286E6F5C
:1005F00020656E74727929000000000000002E2E24
:100600002E2064656C6574696E67202E2E2E002086
:100610006661756C740000000000000000000000BE
:1006200020444343206F6E6C7921000000000000DD
:10063000002A3D43616E63656C20202000000000AD
:1006400000002070726F6772616D696E6700000054
:100650000000002D73686F7274206369726375699E
:10066000742D20002E2E2E207761636874656E2015
:100670002E2E2E2000233D77697373656E000000D7
:10068000000000000000286765656E20696E766FC7
:1006900065722900000000202E2E2E2077697373CA
:1006A000656E202E2E2E000020666F7574000000EF
:1006B00000000000000000000020416C6C65656EC9
:1006C000204443432100000000002A3D204166628F
:1006D00072656B656E0000000000002050726F674D
:1006E00072616D6D6572656E000000002D2D4B6F9F
:1006F0007274736C756974696E672D2D0050617426
:1007000069656E74657A0000000000000000233DFA
:100710007375707072696D6572000000000000767C
:100720006964650000000000000000000000000097
:100730005375707072657373696F6E00000000000E
:100740000020457272657572000000000000000014
:1007500000002044434320756E697175656D656EB8
:100760007400002A3D4162616E646F6E20200000BB
:10077000000000002050726F6772616D6D617469D6
:100780006F6E0000002D436F7572742D6369726384
:100790007569742D20002E2E2E2077617274656E7F
:1007A000202E2E2E202000233D4CF6736368656EAC
:1007B0000000000000000000286B65696E2045699C
:1007C0006E7472616729000000202E2E2E206CF6B8
:1007D00073636865202E2E2E2000204665686C65A8
:1007E0007200000000000000000000206E75722002
:1007F00066FC722044434321000000002A203D2073
:10080000416262727563680000000000002050724F
:100810006F6772616D6D696572756E6700002D2D71
:10082000204B75727A7363686C75DF202D2D005B29
:100830006E6F206D6573736167655D005B756E6BD0
:100840006E6F776E206572726F725D0011241FBE2D
:10085000CFEFD0E1DEBFCDBF11E0A0E0B1E0E8ED29
:10086000FBE400E00BBF02C007900D92A033B1077C
:10087000D9F713E0A0E3B1E001C01D92AA34B1079B
:10088000E1F70C947D040C94000081E08093310129
:100890000895482F90913001981731F0963021F04B
:1008A000953029F4863019F080E090E00895409367
:1008B0003001453021F460E280E00E9450204091F8
:1008C0003001463021F460E280E00E9450200E9416
:1008D000450481E090E008950895809130019927C2
:1008E00008950E94F21D0E94AC108091310188236E
:1008F00011F40E94480BA8950895CFEFD0E1DEBF18
:10090000CDBF0E946F1B0E941D050E944205789476
:100910000E94A2070E94951BFC0184810E94B10BDA
:100920006CEC70E082E00E94D40B0E94AB1B823022
:1009300079F00E94AB1B813059F060E081E00E94A9
:100940005E0A6CED70E082E00E94D40BA895FECFA9
:1009500068ED70E082E00E94D40B60E081E00E94CC
:100960005E0A66E582E00E94B60B6CEE70E082E003
:100970000E94D40B0E94951B8C0181E00E945909B2
:10098000882319F081E00E94981B82E00E94590997
:10099000882319F080E00E94981B83E00E94590987
:1009A000882319F082E00E94981B84E00E94590974
:1009B000882329F083E00E94981B01C0A8950E941B
:1009C000111D8823D9F3F80181859285892BC9F0FF
:1009D0000E94680CEC0146969E012F5E3F4FAC01D1
:1009E000B901F801818592850E945621BC01892BAD
:1009F00029F0F801818592858C8B9D8B611571059D
:100A000019F4F801628173818FEF0E940C1C81E060
:100A100011C00E94C7100E940A0AFFEF8F3F9F0774
:100A2000C1F70E947104809131018823A1F31092D3
:100A3000310180E00E94F50DEECF8FE78ABB1BBA33
:100A400080E187BB18BA80EF84BB8FEF85BB8BEB4F
:100A500081BB8CEC82BB86E082B987EF83B980933F
:100A6000610081EF809362008FE18093640089E1EF
:100A7000809365000E94D308A89588E181BD8CE031
:100A800081BD08950E949D1B9B01AC0193E0E92F5D
:100A9000FF27E45CFE4F822F8F77808387E0569597
:100AA0004795379527958A95D1F7915097FFEFCFC6
:100AB00087B3807F87BB88B3807F88BB84EE8DB986
:100AC00008951F920F920FB60F9211242F933F9308
:100AD0004F935F936F937F938F939F93EF93FF93C6
:100AE00080910001909101018F5F9F4F71F0BB9A3F
:100AF000809100018FB9769B0BC0BB981092320198
:100B0000109239011092380103C0BB988FEF8FB952
:100B10007FB177FF7FC080913A0190913B01892B93
:100B2000E1F0809136018F5F80933601809136012C
:100B3000803210F010923601909136018091370189
:100B4000981759F4809137018F5F80933701809116
:100B50003701803210F01092370180913801909166
:100B600039018F5D924061F058F0809135018F5FBF
:100B70008093350180913501843010F01092350159
:100B800010923B0110923A011092390110923801F3
:100B900060912F01761721F481E08093320171C0BA
:100BA00010923201472F55279A012F773070862FE8
:100BB00099272817390721F07F3F11F06F3F61F423
:100BC0009091360189E0989FC001112481549E4F75
:100BD00090933B0180933A014F775070862F99276D
:100BE0004817590709F04DC09091340180913501A3
:100BF000981749F09091350189E0989FC001112420
:100C000081529D4F02C086EB91E090933901809311
:100C1000380137C020913201822F99278130910508
:100C200031F0813091056CF106975CF516C02F5FAD
:100C300020933201703419F41092330122C07134C0
:100C400011F481E007C0723411F482E003C0733400
:100C500091F483E08093330114C0E22FFF27809149
:100C60003301992702968E179F0744F0E65CFE4FEA
:100C70008081781719F01092320103C02F5F209302
:100C8000320180913201882339F4809138019091AA
:100C90003901892B79F003C0872F99270DC0E09186
:100CA0003801F091390181919927F0933901E0934E
:100CB000380102C08FEF9FEF9093010180930001F4
:100CC00080913A0190913B018F5D924020F010920B
:100CD0003B0110923A01E0913A01F0913B013097CB
:100CE00029F07193F0933B01E0933A01FF91EF916A
:100CF0009F918F917F916F915F914F913F912F9134
:100D00000F900FBE0F901F901895DC018091340159
:100D1000282F332780913501992701972817390704
:100D200041F080913401833039F48091350188237A
:100D300019F480E090E008959091340189E0989F43
:100D4000F0011124E152FD4F98E08D918193915073
:100D500097FFFBCF809134018F5F809334018091A6
:100D60003401843010F01092340181E090E0089555
:100D70000895FC01A6EBB1E098E081918D9391502C
:100D800097FFFBCF08959C01909136018091370128
:100D9000981719F480E090E00895D90121153105E4
:100DA00011F4C9010895F8949091370189E0989F52
:100DB000F0011124E154FE4F98E081918D93915000
:100DC00097FFFBCF809137018F5F80933701809130
:100DD0003701803210F0109237017894C9010895DC
:100DE000089500000000000000000895882341F0ED
:100DF000809165008460809365000E94F1060895EB
:100E0000809165008B7F80936500089508959B0114
:100E1000AC018091050390910603A0910703B09166
:100E2000080382179307A407B507A0F08091050374
:100E300090910603A0910703B0910803821B930BC6
:100E4000A40BB50B80509041A040B040A0F080E0D2
:100E500090E008958091050390910603A091070307
:100E6000B0910803281B390B4A0B5B0B2050304F05
:100E70004F4F5F4F18F081E090E0089580E090E0E0
:100E800008950895EF92FF920F931F93AA27BB270F
:100E9000E0900503F090060300910703109108030A
:100EA000E80EF91E0A1F1B1F01C0A895C801B70153
:100EB0000E9407078823C9F31F910F91FF90EF90BD
:100EC00008950F931F93CF93C82F162F042F80914F
:100ED00065008D7F8093650080E00E94F6068AB3EE
:100EE0008F608ABB8BB3807F9C2F92959F70892BDC
:100EF0008BBB112321F080916500816003C080913C
:100F000065008E7F8093650081E00E94F60680E098
:100F10000E94F606002329F088E090E00E94420734
:100F20000DC08BB3807FCF708C2B8BBB0E94F106E2
:100F300081E00E94F606802F0E94F606CF911F9155
:100F40000F91089588E290E00E94420741E060E03E
:100F500080E30E94610741E060E080E30E94610756
:100F600041E060E080E30E94610741E060E080E2F0
:100F70000E94610788E20E94540A88E00E94540A95
:100F800081E00E94540A86E00E94540A8CE00E948C
:100F9000540A66EC71E080E00E948D0B6EE971E00E
:100FA00081E00E948D0B66EA71E082E00E948D0B69
:100FB0006EE871E083E00E948D0B6EE771E084E0E3
:100FC0000E948D0B66E771E085E00E948D0B6EE656
:100FD00071E086E00E948D0B66E671E087E00E947A
:100FE0008D0B08951F920F920FB60F9211241F932D
:100FF0002F933F934F935F936F937F938F939F9321
:10100000AF93BF93EF93FF9380914201882309F040
:10101000B8C081E0809342017894809140018F5F55
:1010200080934001282F237009F0A9C086958695EA
:101030008770992783309105C1F1843091052CF494
:10104000009759F00197E9F09AC08530910509F4AD
:1010500060C0079709F491C092C0809105039091F8
:101060000603A0910703B09108030196A11DB11DCD
:101070008093050390930603A0930703B09308039E
:101080007EC08091050390910603A0910703B09163
:10109000080381709070A070B070892B19F00E94C5
:1010A0006C096DC00E942D096AC08091410188239E
:1010B00009F465C08AB3807F8ABB822F0E94F6063E
:1010C00080916500826080936500809165008E7FCD
:1010D000809365000000000081E00E94F60619B3CD
:1010E00080E00E94F6061295107F0E94F10681E0D2
:1010F0000E94F60689B38F70182B80E00E94F606D6
:10110000812F992787FD90958827990F881F992708
:1011100031C060914101662391F59091090380915E
:101120000A03981789F010910A03E12FFF27E75F60
:10113000FC4F82811F5F103108F0162F803891F428
:1011400080910903811719F480E090E013C0E12F2A
:10115000FF27E75FFC4F82811F5F103108F0162FD9
:10116000462F02C0462F61E00E94610710930A03D8
:1011700081E090E08093410102C00E94F00910924A
:101180004201FF91EF91BF91AF919F918F917F911C
:101190006F915F914F913F912F911F910F900FBED3
:1011A0000F901F90189510927D0017BE11BE89E612
:1011B00083BF87B7816087BF0895EF92FF920F9337
:1011C0001F93AA27BB27E0900503F0900603009128
:1011D000070310910803E80EF91E0A1F1B1F02C027
:1011E0000E947104C801B7010E9407078823C1F358
:1011F0001F910F91FF90EF900895282F220F6111FA
:101200002160822F83708150823028F424FF02C035
:101210002E6001C0217F822F99270895909145016A
:10122000E92FFF27EB5BFE4F8283892F8F5F80932F
:101230004501883010F0109245019091460180914F
:101240004501981741F4892F8F5F809346018830BC
:1012500010F010924601089508950F931F9311B155
:10126000812F8074682F809143010E94FD08082F10
:10127000809343011078612F809144010E94FD0802
:1012800080934401007C807C003829F4882339F065
:10129000803C61F408C0003449F4803C11F484E1DE
:1012A00003C0882319F485E10E940E091F910F9154
:1012B0000895843118F080E090E0089520E030E057
:1012C000E82FFF27E15BFE4F8081882311F021E0AA
:1012D00030E0C90108950895FF920F931F93CF93B3
:1012E00080916801E82FFF27ED59FE4F008113B36D
:1012F0001083FF2480916801E82FFF27EE0FFF1F66
:10130000EE0FFF1FEF0DF11DEE50FF4FC49110FDCA
:1013100031C000FF14C0C23129F481E10E94590993
:10132000882331F48C2F0E940E09C43108F043C089
:10133000EC2FFF27E15BFE4F81E080833CC0C4318E
:10134000D0F5EC2FFF27DF01A15BBE4F9C919F5F83
:101350009C93992311F49F5F9C937197329758F552
:1013600080916001893738F180916101893718F1E6
:1013700085E01FC0C43128F4EC2FFF27E15BFE4F4E
:10138000108200FD18C08C2F80680E940E090E94F8
:101390006D04853081F4C13121F482E10E94590944
:1013A00005C0C23141F481E10E945909882319F432
:1013B00086E00E94490416950695F39483E08F1504
:1013C00008F098CF809168018F5F80936801853025
:1013D00010F010926801CF911F910F91FF90089526
:1013E00090916801943029F485B3806F85BB9798FC
:1013F0000895979A85B38F7020E130E002C0220FE4
:10140000331F9A95E2F7922F9095907F892B85BB99
:10141000089508958091450120914601821719F49D
:101420008FEF9FEF0895E22FFF27EB5BFE4F828146
:10143000482F5527822F8F5F80934601883010F008
:1014400010924601CA0108950895CF93C82F07C08E
:1014500080910A03882391F40E94F21DA89580913F
:101460000903282F332780910A039927019728170A
:10147000390791F3809109038F3051F3F8948091EB
:101480000903E82FFF27E75FFC4FC2838091090320
:101490008F5F8093090380910903803110F01092CF
:1014A00009037894CF9108951F93182F80E80E9424
:1014B000250A812F0E94250A1F9108958295880F81
:1014C000880F807C860F80680E94540A08950E94CD
:1014D0005E0A8EE00E94540A08958CE00E94540A2D
:1014E0000895FF920F931F93CF93F82E60912C03D2
:1014F00080912B030E945E0AC0E00BE113E0809113
:101500002D03C81778F4FF2021F0F80161918F01B5
:1015100001C060E282E00E94B60BCF5F80912D0394
:10152000C81788F3CF911F910F91FF900895909362
:10153000360380933503892B89F1709334036093CC
:101540003303CB01AA27BB27209105033091060363
:101550004091070350910803280F391F4A1F5B1F52
:1015600020932F0330933003409331035093320381
:1015700080912E038E7F80932E0321153105410526
:10158000510561F42F5F3F4F4F4F5F4F20932F0363
:1015900030933003409331035093320308950895FC
:1015A000AF92BF92CF92DF92EF92FF920F931F9371
:1015B000CF93DF93D82EC62EEA018BE1E82E83E08D
:1015C000F82E109236031092350381E08D1568F1E4
:1015D000EFE0E61750F14115510539F1FA0101909C
:1015E0000020E9F731970E2F041B013108F000E1CC
:1015F0006C2D8D2D0E945E0A5701002361F0102F83
:101600008881F50181935F018991682F82E00E94B2
:10161000B60B1150A9F7F701D08AC18A028B64EF8B
:1016200071E081E79AE00E94970ADF91CF911F91C4
:101630000F91FF90EF90DF90CF90BF90AF90089503
:10164000CF93DF93CDB7DEB7A0970FB6F894DEBF88
:101650000FBECDBF282FDE01119690E0FA014F5F3B
:101660005F4F8491882321F08D939F5F9F31B0F36A
:101670001C92AE014F5F5F4F822F0E94D00AA0964E
:101680000FB6F894DEBF0FBECDBFDF91CF910895A6
:101690008091350390913603892BA9F160912F0336
:1016A0007091300380913103909132030E940707BB
:1016B000882349F180912E03E0913503F0913603A0
:1016C0008170099580912E0391E0892780932E03E4
:1016D00080913303909134039C01442755278091D6
:1016E000050390910603A0910703B0910803820FB0
:1016F000931FA41FB51F80932F0390933003A093D3
:101700003103B09332030895089510923603109276
:10171000350381E00E94540A08950F931F93CF93DD
:10172000DF93EB018830C0F4992723E0880F991FDD
:101730002A95E1F780640E94540A07E010E0FE0158
:10174000219684910E94250A0150104017FFF7CF7F
:1017500060E0862F0E945E0ADF91CF911F910F916A
:101760000895813308F080E381BF08958230D1F479
:1017700067FF15C0643E31F0663F41F06C3F51F0A9
:10178000643C11F461EE0BC0663D11F46FEE07C0CE
:101790006C3D11F465EF03C06F3D09F462EE862FD6
:1017A0000E94250A089508951F93CF93DF93182F61
:1017B000EB01FB016491662349F0812F0E94B60B77
:1017C0002196FE018491682F8823B9F7DF91CF918C
:1017D0001F9108951F93CF93DF93182FEB018881FA
:1017E000882341F08991682F812F0E94B60B888150
:1017F0008823C1F7DF91CF911F9108951F93CF9355
:10180000DF93CDB7DEB7C055D0400FB6F894DEBF3A
:101810000FBECDBF67961FAD679769968EAD9FAD22
:101820006997AE01475A5F4FBC01CE0101960E94F5
:101830007922BE016F5F7F4F812F0E94EA0BC05B50
:10184000DF4F0FB6F894DEBF0FBECDBFDF91CF9153
:101850001F9108951F93CF93DF93CDB7DEB7C05587
:10186000D0400FB6F894DEBF0FBECDBF67961FAD58
:10187000679769968EAD9FAD6997AE01475A5F4FE6
:10188000BC01CE0101960E94A222BE016F5F7F4F74
:10189000812F0E94EA0BC05BDF4F0FB6F894DEBFCA
:1018A0000FBECDBFDF91CF911F910895823019F403
:1018B0000E940A0A08958FEF9FEF08950895E82F78
:1018C000FF27EF70F070E25EFD4F84919927089535
:1018D00089E691E008958091790182FF05C08091A9
:1018E0006B0190916C0108958091690190916A015A
:1018F0000895089580917901826080937901089517
:101900000F931F93CF93DF93C9E6D1E080917901C4
:1019100099278C010170107080FF03C080E090E077
:1019200021C0609171017091720180917301909159
:101930007401611571058105910531F00E94070759
:10194000882311F4C8010EC01A821B821C8A1D8ACA
:1019500010926A0110926901188A1E8A0E94450439
:1019600081E090E0DF91CF911F910F9108959C014C
:1019700080916B0190916C01892B11F4C90108953C
:101980002F703F7B77FD3064CB018F70907044E007
:10199000880F991F4A95E1F7822B932B089508959C
:1019A000FC018091690190916A0120916B01309155
:1019B0006C01E817F907F9F460937B01232BB1F070
:1019C00080916F0190917001F4E096958795FA955A
:1019D000E1F7BC016F707070892F99278695869505
:1019E00080FD7068CA010E94B70C0FC0509370014F
:1019F00040936F010EC0E217F30769F4BA018091BA
:101A00006F01909170010E94B70C909370018093C8
:101A10006F010E944504089508959C01892B69F483
:101A2000109279011092710110927201109273015B
:101A3000109274010E94800C089560937B01509372
:101A4000700140936F018091050390910603A0916E
:101A50000703B091080388519C4FAF4FBF4F81607F
:101A60008093710190937201A0937301B0937401FC
:101A70008091790182FF09C081608B7F8093790119
:101A800030936C0120936B0107C08E7F80937901A6
:101A900030936A01209369010E94450408950895D6
:101AA000209179012B7F21602093790190936C0123
:101AB00080936B0180916F01909170010E94B70C2F
:101AC0009093700180936F010E9445040895CF9315
:101AD000DF93EB0180937A010E945F0C80937C017D
:101AE000209759F04FE751E060E070E0CE010E948E
:101AF0005621D0937E01C0937D010E944504DF9161
:101B0000CF910895CF93C82F882319F06EE571E027
:101B100002C06EE771E084E00E948D0BCC2319F0C7
:101B200066E571E002C066E771E085E00E948D0B1A
:101B3000CC2319F06EE471E002C06EE671E086E03D
:101B40000E948D0BCC2319F066E471E002C066E6BA
:101B500071E087E00E948D0BCF910895CF93DF93C2
:101B6000C82FDD27C4FF02C083E001C085EA0E94C0
:101B7000250AC0FF02C084E001C085EA0E94250A50
:101B8000C1FF02C085E001C085EA0E94250AC2FFAC
:101B900002C086E001C085EA0E94250AC3FF02C098
:101BA00087E001C085EA0E94250ADF91CF91089560
:101BB00080938B010E9445040895882319F066E202
:101BC00071E002C06EE271E082E00E948D0B089528
:101BD0000895882319F066E371E002C06EE371E0B6
:101BE00081E00E948D0B089508950F931F93CF936A
:101BF00009E611E0C0918B01CC2399F060E081E00F
:101C00000E945E0A8C2F81500E94171BBC0182E04B
:101C10000E94D40B10928B0188EE93E00E94DD08A5
:101C200002C0882319F00E94850B03C0682F0E9410
:101C30005E0A8091690190916A01892BF9F00E94F6
:101C4000951BFC01828193814091690150916A0149
:101C50008417950749F42185328580917D01909103
:101C60007E012817390751F04283538380917D010B
:101C700090917E01818792870E943A1B2091690191
:101C800030916A012115310529F4F8012683378343
:101C9000128A118A8091790182FD0DC080917501AF
:101CA00090917601A0917701B09178010097A105FC
:101CB000B10519F105C06EE272E082E00E94D40B1A
:101CC0008091750190917601A0917701B091780192
:101CD000BF93AF939F938F9381E392E09F938F93F2
:101CE00082E08F930E942A0C8DB79EB707960FB69D
:101CF000F8949EBF0FBE8DBF43C02115310531F44E
:101D000064E472E082E00E94D40B18C03F932F93EA
:101D10008BE492E09F938F93C2E0CF930E942A0CB2
:101D2000809179010F900F900F900F900F9080FF8E
:101D300002C08C2F01C080E20E94250AC0917A0166
:101D40000E946D04853010F085E00EC0833061F490
:101D50008C2F99278370907023E0880F991F2A9504
:101D6000E1F782539E4F08C0992703E0880F991F1F
:101D70000A95E1F782519E4FBC0182E00E94D40B8C
:101D80006CE080E00E945E0A80917B0199278F774A
:101D900090709F938F9380E592E09F938F9382E062
:101DA0008F930E942A0C80917A01992783709070FA
:101DB0000F900F900F900F900F90019779F483E19F
:101DC0000E945909882331F080E00E94250A6EE0C4
:101DD00071E010C080E20E94250A0FC080E00E94DE
:101DE000250A80917B0187FF03C066EC71E002C089
:101DF0006EEB71E080E00E948D0B0E946D04C82F95
:101E0000813049F488E00E94E21AAC0160E08C2F36
:101E10000E94200BE0C040E050E060E0862F0E946E
:101E2000D00AC0E08AE00E945909882371F08091AD
:101E30006B0190916C01892B39F480917A0199277B
:101E400083709070039709F4C1E060E081E00E9424
:101E50005E0A8091750190917601A0917701B09111
:101E600078010097A105B10509F442C08DE00E94F8
:101E70005909882329F48EE00E945909882381F1A9
:101E800084E592E09F938F93C2E0CF930E942A0C47
:101E90008DE00E9459090F900F900F90882379F0E0
:101EA00066E371E081E00E948D0B6EE271E08C2FA1
:101EB0000E948D0B6CE271E089EE9DE00EC06EE336
:101EC00071E081E00E948D0B66E271E08C2F0E9430
:101ED0008D0B6CE271E08DED9DE00E94970A7BC056
:101EE00086E00E94E21ABC0182E00E94D40B44C04A
:101EF00080916B0190916C01009769F19F938F9392
:101F000080E692E09F938F9382E08F930E942A0C49
:101F100080916F019091700114E0969587951A95C4
:101F2000E1F7282F2F70892F9927869586950F9096
:101F30000F900F900F900F9080FD2061822F0E94D4
:101F4000AE0DCC2321F08CE30E94250A15C080E25F
:101F50000E94250A2CC08FE791E09F938F9385E61E
:101F600092E09F938F9382E08F930E942A0C0F90B0
:101F70000F900F900F900F90CC23C9F080916B01C0
:101F800090916C01892B99F480916F01909170016F
:101F9000A4E096958795AA95E1F78F7080610E94DD
:101FA000AE0D81E00E94820D66E871E011C02091C3
:101FB0006F012F7080916F019091700197FD2061EA
:101FC000822F0E94AE0D80E00E94820D6EE871E0CB
:101FD00083E00E948D0BCF911F910F910895EF9296
:101FE000FF920F931F93CF93DF93CDB7DEB7269762
:101FF0000FB6F894DEBF0FBECDBF8C0186E0FE01A8
:10200000319611928A95E9F7F80124853585468540
:10201000578562817381211531054105510509F408
:1020200083C06115710569F1E080F180C701AA27BD
:10203000BB2782179307A407B50741F0CB01AA2756
:10204000BB2782179307A407B507D9F4F801808945
:102050008E7F808B80818F778983EE0CEF2CEE1C36
:10206000FF08F1948E2D8F778A83AE014F5F5F4F0B
:1020700065E080E00E94DC1DF8011282138210826C
:102080001182D8018D919C919C0144275527F8011C
:1020900084859585A685B7856089281739074A07FD
:1020A0005B0729F481E068276B7F608B44C06C7FFD
:1020B000F801608B148A158A168A668981E00E946D
:1020C0005E0A80E00E94E21ABC0182E00E94D40B0A
:1020D000F8018089992796958795969587959C0113
:1020E0002170307080FD14C080819181009711F0C3
:1020F00084839583F8012283338326833783208367
:102100003183118A648575858FEF0E940C1C08C08D
:10211000F80144855585608171818FEF0E943B1CD9
:10212000F80180898B7F05C0672B21F4F801808935
:102130008460808BF801148615861686178626968D
:102140000FB6F894DEBF0FBECDBFDF91CF911F91C8
:102150000F91FF90EF90089560917101709172015D
:10216000809173019091740161157105810591054C
:1021700061F00E940707882341F0109271011092CC
:102180007201109273011092740108950895AF9234
:10219000BF92CF92DF92EF92FF920F931F93CF9354
:1021A000DF93CDB7DEB72C970FB6F894DEBF0FBE26
:1021B000CDBF8C0129E6C22E21E0D22E86E0FE01A1
:1021C000319611928A95E9F701311105DCF40F304F
:1021D00011050CF0EFC00A30110509F479C10B307C
:1021E00011053CF40115110509F410C117FD7FC15B
:1021F0003AC10C30110509F460C00D3011050CF026
:102200007BC061C105311105C1F1063111057CF4B6
:102210000231110509F4EAC0023111050CF4E8C0DD
:1022200003311105B9F10431110591F060C10F3886
:1022300011054CF40D3811050CF05EC00A3811057B
:1022400009F453C154C10339110509F44EC14FC1FA
:1022500080917B0199278F77907020917C013327A3
:10226000821793070CF043C10E946D04833009F07C
:102270003EC180917B018F5F1DC020917B01822F29
:1022800099278F779070892B09F431C121502093C1
:102290007B012BC180917A019927837090700197FF
:1022A00029F46EE071E080E00E948D0B80917B014B
:1022B0008095807880937B0118C18AE00E9459093B
:1022C000882399F080916B0190916C01892B69F0C2
:1022D00080916F019091700120E030E48227932774
:1022E0009093700180936F0100C180916F01909174
:1022F000700120E030E874C086E097E0A92EB12C90
:10230000AC0EBD1EF50111928A95E9F78091750119
:1023100090917601A0917701B09178010097A10585
:10232000B10509F445C0E0907501F090760108947C
:10233000E108F108EE0CFF1CC8018F7790700E9732
:1023400021F481E090E0E82AF92A07FF16C01A86F6
:1023500060E070E0CB010E94970A6EE971E081E0D5
:102360000E948D0B66EA71E082E00E948D0BF601FF
:10237000148615861686178602C081E08A878E2D00
:102380008F778F83EE0CEF2CEE1CFF08F1948E2DCF
:102390008F778887EE0CEF2CEE1CFF08F1948E2DC2
:1023A00083708987A50166E080E00E94DC1D9DC0E6
:1023B00007FD9BC0E3EFFE2EF00E8AE00E94590954
:1023C000882319F077EFF72EF00E21E030E002C0FD
:1023D000220F331FFA94E2F780916F019091700100
:1023E00082279327F601868397837FC043E006C048
:1023F0008AE00E945909882321F042E060E280E0EF
:1024000002C0482F60E20E9450206FC08AE00E9404
:1024100059098823A9F080916D0190916E01009770
:1024200009F465C0AA27BB278093750190937601B4
:10243000A0937701B0937801C6010E94EF0F57C0B7
:102440008091750190917601A0917701B09178010A
:102450000097A105B10539F48FEF0E94B01A81E011
:102460000E94F50D44C08091750190917601A09174
:102470007701B09178019C01AD0163E0220F331F19
:10248000441F551F6A95D1F7280F391F4A1F5B1F3C
:10249000280F391F4A1F5B1FC801AA2797FDA09567
:1024A000BA2F280F391F4A1F5B1F2030F8E23F0761
:1024B000F0E04F07F0E05F07D4F4F601248735879A
:1024C0004687578712C089E691E00E94EF0F0DC042
:1024D0001092750110927601109277011092780196
:1024E000809179018B7F809379010E9445042C961D
:1024F0000FB6F894DEBF0FBECDBFDF91CF911F9115
:102500000F91FF90EF90DF90CF90BF90AF90089524
:10251000FB0121E057FF04C020E0509541955F4F3B
:102520008330910549F18430910534F4813091056F
:1025300091F0029729F12AC08430910519F005978E
:1025400061F024C081818F5F81839927841795076B
:10255000ECF0222359F0118219C0818181508183CE
:1025600099278417950794F0222321F0842F815016
:1025700081830CC021830AC012821382168A06C08E
:1025800090E08281882309F491E0928380E090E0DA
:1025900008950F931F93CF93DF938C010E946B0CD0
:1025A000EC01009731F469E375E082E00E94D40BFE
:1025B0000FC09F938F938FE395E09F938F9382E05B
:1025C0008F930E942A0C0F900F900F900F900F90F6
:1025D0000115110521F0B80182E00E94D40BCE0153
:1025E000DF91CF911F910F9108950F931F93CF9378
:1025F000DF93EC018B01009731F097FD35C0029716
:10260000029790F52BC060E081E00E945E0AF8011D
:102610008281882359F463E475E082E00E94D40B40
:102620006CE475E082E00E94D40B18C00E949D1BF0
:10263000DC01CB01BF93AF939F938F9382E595E02D
:102640009F938F9382E08F930E942A0C8DB79EB741
:1026500007960FB6F8949EBF0FBE8DBF40E050E0C6
:10266000B801CE010E94881280E090E0DF91CF9106
:102670001F910F9108958230910541F083309105AB
:1026800041F440E050E00E94881203C08FEF9FEFBA
:10269000089580E090E0089508952F923F924F9220
:1026A0005F926F927F928F929F92AF92BF92CF92E2
:1026B000DF92FF920F931F93CF93DF93CDB7DEB7D7
:1026C00026970FB6F894DEBF0FBECDBF8C015B011D
:1026D0000E94680C6C010230110509F457C00330E8
:1026E00011053CF401151105E9F00130110531F037
:1026F000CAC0063011050CF0C6C02CC0FC01F18820
:102700002F2D269526952370F3E0FF2211F451E03A
:10271000F52E83E0F89EC0011124280F2350F50107
:102720002183B1C060E081E00E945E0A8EE595E001
:102730000E94C912892B09F4A6C0F50191818AE093
:10274000989FC001112481569D4FBC0182E00E94D8
:10275000D40B99C049E050E0B501C8010E9488122D
:10276000F601808191818F3F910509F008F48BC0BB
:10277000F5018181882311F486E08183F50181814F
:10278000863008F080C088E081837DC0FC014280F3
:1027900053804114510409F076C0F50182818823E9
:1027A00009F469C0F601808091808114910409F4D4
:1027B0006AC0F5012181822F63E00E94BE25F82EB8
:1027C000F394822F0E94BE25892F9927880F991F85
:1027D000880F991FF82AF6012488358836E1632E80
:1027E000712C6C0C7D1C8501065F1F4FB301C80165
:1027F0000E94722286E0FE01319611928A95E9F7D5
:10280000882D8F778983C401880F892F881F990BA2
:1028100091958F778A83FFE7FF22FB82AE014F5F9E
:102820005F4F64E08FEF0E94DC1D60E081E00E945A
:102830005E0A80E00E94E21ABC0182E00E94D40B92
:10284000A20160E0C2010E940D0DB4018FEF0E9451
:102850000C1CB801C3010E9472222114310459F0EA
:102860009301F601418960817181C1010E94992023
:10287000F601848B958B90E0F5018281882309F421
:1028800091E0F501928380E090E026960FB6F894EF
:10289000DEBF0FBECDBFDF91CF911F910F91FF9093
:1028A000DF90CF90BF90AF909F908F907F906F9070
:1028B0005F904F903F902F900895482F30E0832FE6
:1028C000992787FD9095FC01E259FD4F249124172B
:1028D00029F03F5F222399F78FEF9FEF0895089526
:1028E000EF92FF920F931F93CF93DF93EB01823010
:1028F000910509F486C08330910534F4009709F4FA
:102900003EC0019769F0BAC08430910509F443C014
:10291000843091050CF470C0059709F456C0AEC020
:102920000E94680C8C01FC0180819181892B09F443
:10293000A5C066E1E62EF12CE00EF11E8E01065FC9
:102940001F4F65960C171D07B8F4F7018081882387
:1029500039F00E945D1487FD03C0F701808101C03A
:1029600080E2F80181938F01F7018081882351F380
:102970000894E11CF11CE6CFF80110827FC00E9490
:10298000C91260E081E00E945E0A2A96BE0182E0E0
:102990000E94EA0B73C08981FB01E80FF11DEF0172
:1029A0002A9682850E945D148F5FE82FFF27E7FD3E
:1029B000F095E259FD4F8491882319F4EEE6F2E098
:1029C0008491992787FD909515C08981FB01E80FB7
:1029D000F11DEF012A9682850E945D14181614F0ED
:1029E0008FE201C08150E82FFF27E7FDF095E25903
:1029F000FD4F8491888342C049E050E00E948812D4
:102A00003DC00E94680C8C01FC0182819381892B5E
:102A1000A9F59A81992349F489E08B8381E0888F15
:102A200099839F8B8A838E8B29C089818F5F89834D
:102A30008F8B8B3018F11B821A821E8A8CE09801D2
:102A40002A5E3F4FD901FE013A9601900D928A9578
:102A5000E1F7F80184899589009731F04189608117
:102A600071810E94992007C0A901F80161898081C4
:102A700091810E944E21F801848B958B80E090E03B
:102A8000DF91CF911F910F91FF90EF9008958F925A
:102A90009F92BF92CF92DF92EF92FF920F931F937C
:102AA000CF93DF93CDB7DEB727970FB6F894DEBF8D
:102AB0000FBECDBF9C018B018230910509F455C03A
:102AC000833091052CF40097C1F0019759F0C8C0EC
:102AD00084309105D9F1843091050CF441C00597FB
:102AE000C9F1BEC04BE050E060E270E0C8010A9658
:102AF0000E946B22F801158AB3C0FB0182818823F2
:102B000009F4AEC08181882309F4AAC0065F1F4F73
:102B1000A801B90199270E9456219F938F9381E6BE
:102B200095E09F938F93F2E0FF2EFF920E942A0C74
:102B300060E081E00E945E0AB8018F2D0E94EA0BDE
:102B40000F900F900F900F900F908AC0FB01818122
:102B5000992721C0FB01818199270E9443221DC032
:102B600049E050E00E9488127BC090E0FB01828126
:102B7000882309F491E0F80192830E94680C7C019B
:102B8000F801B280BB2061F0FC018489958900972F
:102B900011F0848902C00E943F22F801818360C045
:102BA000EAE08E2E912C800E911EF8018181A40105
:102BB000BE01695F7F4F99270E9456216C01F70182
:102BC0001282138210821182BC018FEF0E940C1CB2
:102BD000F70180819181892B81F186E0FE01319698
:102BE00011928A95E9F78C2D8F778983C601880F1A
:102BF000892F881F990B91958F778A838F818F7783
:102C00008B83AE014F5F5F4F64E08FEF0E94DC1D4E
:102C10006B2D81E00E945E0A8B2D0E94E21ABC019E
:102C200082E00E94D40B40E050E06B2DCA010E946C
:102C30000D0DB6018FEF0E940C1CF7018081918170
:102C4000892B59F0B401C70146960E947222F801FF
:102C500081819927F701848B958B8FEF9FEF02C0BD
:102C600080E090E027960FB6F894DEBF0FBECDBF90
:102C7000DF91CF911F910F91FF90EF90DF90CF9058
:102C8000BF909F908F9008950F931F93CF93DF93E2
:102C9000EC010E94680C8C01209719F02297C9F072
:102CA0003DC0CE010E94C912892BC1F160E081E0D4
:102CB0000E945E0AF80184899589892B11F081E0D0
:102CC00001C082E00E94E21ABC0182E00E94D40BA3
:102CD00025C0FC01C281D381209701F580819181BB
:102CE000892BE1F084899589892BC1F060E081E02E
:102CF0000E945E0A83E00E94E21ABC0182E00E9408
:102D0000D40B84EF91E00E94DD08F8018489958955
:102D10000E946F20F801C48BD58B168A80E090E06A
:102D2000DF91CF911F910F9108951F93CF93DF9360
:102D3000EB018230910509F440C0833091052CF4F9
:102D4000009789F0019731F04CC0863091050CF066
:102D500048C02EC00E94951BFC01848163E00E9444
:102D6000BE2589833EC060E081E00E945E0A8981C1
:102D700013E0819F802D11240E94B10B82E090E02E
:102D80000E94DD0881B7612F0E94BE2589839927A3
:102D90009F938F9385E695E09F938F9382E08F9327
:102DA0000E942A0C0F900F900F900F900F9019C057
:102DB0004FEE5FEF0E94881214C08A81882359F079
:102DC0000E94951B398123E0329F90011124FC0160
:102DD00024830E943A1B90E08A81882309F491E0C1
:102DE0009A8380E090E0DF91CF911F910895EF9258
:102DF000FF920F931F93CF93DF93CDB7DEB7269744
:102E00000FB6F894DEBF0FBECDBF8C017B010E94D0
:102E1000680CDC018D919C911197892B39F0FD0193
:102E20008189992783709070039731F060E081E089
:102E30000E945E0A85E03AC00230110509F4A3C081
:102E4000033011053CF40115110539F1013011056C
:102E500071F0F8C00430110509F493C00430110575
:102E60000CF4EAC00530110509F4E2C0EBC08EEFA6
:102E70009FEFF701818F928F209193013091940100
:102E8000C90101978050944020F4F70124833583D1
:102E9000D9C0F70104831583D5C060E081E00E94AA
:102EA0005E0AF7018281882341F487E00E94E21ADA
:102EB000BC0182E00E94D40BC5C060E081E00E94AA
:102EC0005E0AF701848195819F938F9389E695E04F
:102ED0009F938F9312E01F930E942A0C0F900F90E4
:102EE0000F900F900F90F7018381843059F48FE693
:102EF00095E09F938F931F930E942A0C0F900F9041
:102F00000F9011C0F701808599279F938F9383E7D6
:102F100095E09F938F931F930E942A0C0F900F9020
:102F20000F900F900F90F701818D928D97FD03C048
:102F300067E775E00AC08E5F9F4F19F46FE775E091
:102F400004C084E00E94E21ABC0182E00E94D40B1B
:102F500081E0F701808F868B8381992781309105ED
:102F60006CF08330910524F00497029738F402C086
:102F700083E001C088E0F701878B64C0F701168AFF
:102F800061C084E056C0F7018281248135818823A5
:102F900089F441E0438380E094E08683978382173D
:102FA00093072CF481E090E0F70184839583F70187
:102FB000428348C030939401209393012115310539
:102FC000B9F1F70183818150823090F18C918F7734
:102FD00089838D919C91880F892F881F990B9195DA
:102FE0008F778A83848181508F778B832150304003
:102FF000220F232F221F330B322F37702085822F71
:1030000099278078907095958795382B3C832F77FA
:103010002D831E82AE014F5F5F4F67E08FEF0E94EE
:10302000DC1DF70113820E946D0A8FEF9FEF0CC029
:1030300081E0F701838306C040E050E0B701C8019A
:103040000E94881280E090E026960FB6F894DEBFCA
:103050000FBECDBFDF91CF911F910F91FF90EF90E9
:103060000895CF92DF92EF92FF920F931F93CF9329
:10307000DF937C01C62F0E94850B0E94951B6C017B
:10308000CA3008F06FC085E0C89F800111240E5F30
:103090001E4FF7018281882311F080E001C082E099
:1030A0000E94250AF6018581992781309105B1F0AA
:1030B000823091051CF4892B39F031C082309105A2
:1030C000B9F00397F9F02BC08C2F992754E0880FA3
:1030D000991F5A95E1F787559B4F1DC08C2F992753
:1030E00044E0880F991F4A95E1F7875E9B4F13C014
:1030F0008C2F992734E0880F991F3A95E1F787576D
:103100009C4F09C08C2F992724E0880F991F2A957E
:10311000E1F787509D4FBC0182E00E94D40BE8018B
:103120008C8187FD0BC060E081E00E945E0A8C818B
:103130000E94E21ABC0182E00E94D40BE801EA81FD
:10314000FB81309721F0B70180E090E00995F7010D
:103150008689882329F06789808D0E94670A02C0CA
:103160000E946D0ADF91CF911F910F91FF90EF9018
:10317000DF90CF90089560E0E2E0F1E0482F55271E
:1031800047FD509520E030E080819927841795070E
:1031900011F4C90108956F5F2F5F3F4F3596693075
:1031A00098F38FEF9FEF08950895BF92CF92DF922B
:1031B000EF92FF920F931F93CF93DF93CDB7DEB7BC
:1031C0006B970FB6F894DEBF0FBECDBFB82E28E0C8
:1031D000281718F480E090E0B3C16E010894C11C78
:1031E000D11C8BE1F60111928A95E9F7A89585E04B
:1031F000B89EF0011124EE5FFE4F0280F381E02DB6
:10320000309721F0B60181E090E009956B2DC60161
:103210000E9431180E94710415E0B19E70011124C2
:1032200082E091E0E80EF91E0E940A0AAC018B30A0
:10323000910509F497C08C30910534F497FDEACFDD
:103240000A970CF4FEC0D6C08331910509F48AC0F8
:103250008431910524F4419709F46BC1DBCF8431AB
:10326000910519F0459751F1D5CFF6018281882358
:1032700081F0F701228133812115310531F0BE0142
:103280006F5F7F4F84E090E051C1F60181818F5FD5
:1032900028C0F601868BF7019081F7E0FB1534F02A
:1032A000F7018581891711F4B39431C0892F0E94E9
:1032B000BB18682F772767FD709540C0F6018281A3
:1032C000882389F0F701228133812115310531F0FE
:1032D000BE016F5F7F4F85E090E028C1F6018181DC
:1032E0008150818329C1F601868B6B2DF701908176
:1032F000BB2091F02BEF3FEFE20EF31EF701808130
:1033000025E030E0E20EF31E891731F4BA946B2DFC
:10331000772767FD709512C037E03B1564F0D70141
:103320001596F7018581891731F46F5F68301CF4B9
:1033300015968C91F8CF772767FD7095B62E85E0AE
:10334000689FF0011124EE5FFE4F0280F381E02DB3
:10335000309709F4F1C0BE016F5F7F4F81E090E0CC
:103360000995EAC0F7019181992361F1092F11278D
:1033700004571E4FF801808118162CF0892F0E94E7
:10338000BB18F8018083F7018181E82FFF27E457FC
:10339000FE4F80810E94D518282F332727FD3095B6
:1033A000F7018181E82FFF27E457FE4FC90137FF5E
:1033B00004C088279927821B930B808337FFBCC0EA
:1033C000B1943AC0F701228133812115310551F0C2
:1033D000BE016F5F7F4F82E090E0F901099599236C
:1033E0007CF319C0F6018281882309F491E0F6018B
:1033F0009283A2C0F60182818823F1F0F701228135
:10340000338121153105A9F0BE016F5F7F4F83E045
:1034100090E0F9010995F6018281882309F08CC0BA
:10342000F70122813381BE016F5F7F4F81E090E021
:103430007DC0F601128280C08B2D992787FD909563
:103440007FC0F601838199278430910509F446C035
:10345000853091054CF48230910539F18330910526
:1034600084F4019771F068C08830910551F089307B
:1034700091051CF40597A9F15FC0099709F444C0B0
:103480005BC0F60186819781892B21F48FEF9FE73E
:1034900086839783F60186819781841795070CF4BC
:1034A0004BC01482158282E08383F601848195816A
:1034B0009C0163E0220F331F6A95E1F7280F391F43
:1034C000280F391F240F351F37FD36C0868197819D
:1034D000821793078CF1248335832EC0F601108662
:1034E0001383F60190858AE0989F90011124240FA0
:1034F000351F2F3F310509F008F420878EEF9FEF2D
:10350000F601818F928F18C0F6018181E80FF11DBD
:10351000842F805D8287F701228133812115310557
:1035200059F0BE016F5F7F4F82E090E0F90109958D
:1035300003C080E00E9449046B2DCE01019668CE45
:103540006B960FB6F894DEBF0FBECDBFDF91CF9163
:103550001F910F91FF90EF90DF90CF90BF90089553
:10356000CF93C82F66E071E080E00E948D0B6EE083
:1035700071E082E00E948D0B80918C01893010F007
:1035800010928C01C7FD04C08C2F0E94D5180EC06C
:1035900080918C010E94D518992787FD909597FFFF
:1035A00003C0909581959F4F80938C0166EC71E0EC
:1035B00080E00E948D0B66EA71E082E00E948D0B34
:1035C000CF910895CF93C82F893018F08FE298E0FB
:1035D0002CC00E94951BFC018581992782309105A2
:1035E00081F0833091051CF4019721F018C00397F6
:1035F00079F015C081E1C89FC00111248A56984F07
:1036000014C081E1C89FC00111248350994F0DC09F
:1036100081E1C89FC00111248C59994F06C081E1F6
:10362000C89FC001112485539A4FCF9108958823D4
:1036300019F08CE398E008950E94951BFC018581A8
:1036400099278230910561F0833091051CF4019730
:1036500021F00CC0039739F009C08AEB95E008957A
:1036600089EA95E0089588E995E0089587E895E06E
:1036700008950895EF92FF921F93CF93DF9385E90A
:10368000E82E81E0F82EC0E0D0E01FE1CE010E94DC
:103690004722F70161917F01861719F0CE010E9440
:1036A0006022A8951150219617FFF0CFDF91CF919E
:1036B0001F91FF90EF90089590919A01943008F037
:1036C00091E08FE0E5E9F1E011928A95E9F788E170
:1036D0008093990190939A010E943A1B089540E2C9
:1036E00050E060E070E085E991E00E944F22809117
:1036F0009701909198018F5F9F4F11F40E945C1B7E
:1037000080919A01843010F010929A018AEF9FEF15
:10371000A1E0B0E0ABBFFC0187918F3F21F088238F
:1037200011F080936F000895089585E991E0089560
:1037300080939A010E943A1B08958CEF9FEFA1E0BD
:10374000B0E0ABBFFC0187919791A791B691B070A3
:10375000BC01CD0108958FEF9FEFA1E0B0E0ABBFBA
:10376000FC01879199270895FC01808999279695F6
:1037700087959C012170307080FD02C0C9010895B9
:1037800080819181009711F081E090E00895089583
:10379000FC0182819381009711F081E090E008950F
:1037A0000895CF92DF92EF92FF920F931F93CF93E2
:1037B000DF93C82E7B01EA010E94680C8C012097E0
:1037C00011F1DD24A7016C2D80E00E94DC1D8AE050
:1037D0008093370302C00E947104C801FE0109955D
:1037E000882321F4809137038823A9F70E94041DC0
:1037F0008111DD24C801FE010995882321F4D394A9
:1038000087E08D15F8F6DF91CF911F910F91FF9012
:10381000EF90DF90CF900895CF93DF93CDB7DEB7D1
:1038200026970FB6F894DEBF0FBECDBF61157105A8
:10383000C9F086E0FE01319611928A95E9F7862F4C
:103840008F778983660F672F661F770B7195862F99
:103850008F778A8344EB5BE1BE016F5F7F4F81E02E
:103860000E94D11B26960FB6F894DEBF0FBECDBFC7
:10387000DF91CF910895CF93DF93CDB7DEB7269731
:103880000FB6F894DEBF0FBECDBF6115710539F1DB
:103890004115510521F186E0FE01319611928A957C
:1038A000E9F7862F8F778983660F672F661F770B5F
:1038B0007195862F8F778A83842F8F778B83440F20
:1038C000452F441F550B5195842F8F778C8348ECDF
:1038D0005BE1BE016F5F7F4F82E00E94D11B2696A5
:1038E0000FB6F894DEBF0FBECDBFDF91CF91089524
:1038F000F894FFCFFC0180E0482F57E02191282762
:1039000080E0922F96958F5F20FF03C0292F2527F7
:1039100001C0292F8830A8F33327822F4F5F48300A
:1039200068F327FD8095992708950F931F938C01C5
:103930000E947A1CF8019085891719F080E090E0C8
:1039400002C081E090E01F910F910895EF92FF92E5
:103950000F931F93CF93DF93CDB7DEB729970FB6A1
:10396000F894DEBF0FBECDBF9C0180912F0180680F
:103970007E010894E11CF11C898383E0F7018183B7
:1039800087010E5F1F4F822F8F77F8018193220FDF
:10399000232F221F330B3195822F8F778193862F10
:1039A0008F7781938F01CA01892F992786958695F4
:1039B0008F73808367FF02C0806480830F5F1F4F17
:1039C000CA0123E0969587952A95E1F78F77F8014C
:1039D0008193842F8295807F8F7781938F01C70198
:1039E0000E947A1CF8018083C7010E94B9062996BB
:1039F0000FB6F894DEBF0FBECDBFDF91CF911F9100
:103A00000F91FF90EF9008958091B501882319F4EC
:103A100080E090E008951092B50181E090E0089573
:103A20000895EF92FF920F931F93CF93DF93CDB73B
:103A3000DEB729970FB6F894DEBF0FBECDBF0E9448
:103A40009D1B7B018C0165C0A8958A81843009F09B
:103A500060C0CE0101960E94951C882309F459C0CC
:103A6000D801C7018F779070A070B0702E81332776
:103A70004427552782179307A407B50709F049C0C3
:103A8000D801C70180789F73A070B07027E0B5950A
:103A9000A795979587952A95D1F72D8133274427A8
:103AA000552782179307A407B50799F5D801C701D1
:103AB0008070907CAF71B070FEE0B595A79597953A
:103AC0008795FA95D1F72C813327442755278217FC
:103AD0009307A407B507E9F4D801C7018070907077
:103AE000A07EB070E5E1B595A79597958795EA9585
:103AF000D1F72B8133274427552782179307A40733
:103B0000B50739F489818F7780932F0181E090E0A8
:103B100007C0CE0101960E94C306009709F094CF1A
:103B200029960FB6F894DEBF0FBECDBFDF91CF91BF
:103B30001F910F91FF90EF90089580912F01992789
:103B400008950F931F93CF93DF93CDB7DEB72997D7
:103B50000FB6F894DEBF0FBECDBFFA01A8958091D5
:103B60002F01806889836A838E010D5F1F4F95E066
:103B7000309729F081918F77D8018C9302C0D801BA
:103B80001C9291500F5F1F4F97FFF2CFCE0101960D
:103B90000E947A1CF8018083CE0101960E9485065E
:103BA000992729960FB6F894DEBF0FBECDBFDF91DF
:103BB000CF911F910F9108950F931F93CF93DF9390
:103BC000082F162FEA0102C00E947104AE01612F76
:103BD000802F0E94A11D8823B9F3DF91CF911F91FF
:103BE0000F9108959F92AF92BF92CF92DF92EF9282
:103BF000FF920F931F93CF93DF93CDB7DEB72F972D
:103C00000FB6F894DEBF0FBECDBF31C2CE01019614
:103C10000E94951C882309F42AC26E010894C11CD5
:103C2000D11C0E94680C5C01F6016181862F9927E6
:103C3000AA27BB27FC013397E032F10508F0EDC15C
:103C4000EA5BFF4FEE0FFF1F0590F491E02D099402
:103C5000F60182810E944904E0C1F6018281282F89
:103C60003327838199279695982F8827979587954D
:103C7000282B392BD5018D919C918217930709F040
:103C8000CCC10E94800CC9C1F6018281A82FBB273C
:103C9000838199279695982F882797958795A82BA4
:103CA000B92B8581282F3327A901542F4427550F7D
:103CB000550F868199278F77907013E0880F991F91
:103CC0001A95E1F7482B592B8781992780779070B7
:103CD00074E0959587957A95E1F7482B592B6830D4
:103CE00029F4BA01CD010E94500D97C1F6016481FB
:103CF00026FD6068CD010E940D0D8FC1F601858102
:103D0000282F3327868199279695982F882797956E
:103D10008795282B392BB90184810E94670D7DC1BD
:103D20000E947A0C7AC1F6018281A82FBB27838179
:103D300099279695982F882797958795A82BB92B23
:103D40008581282F3327A901542F4427550F550F5C
:103D5000868199278F77907003E0880F991F0A95C5
:103D6000E1F7482B592B878199278077907014E0D1
:103D7000959587951A95E1F7482B592B648126FD77
:103D80006068CD010E94D00C48C1F50184899589F5
:103D9000892B41F0A8E09A2E84898F778A878489BD
:103DA000958907C09924D5018C918F778A878D9149
:103DB0009C91880F892F881F990B91958F778B87FE
:103DC000F501808980FF02C0F0E19F2A0E949D1BBF
:103DD0007B018C01862F8F778C8767E0169507957E
:103DE000F794E7946A95D1F78E2D8F778D8757E0FA
:103DF00016950795F794E7945A95D1F78E2D8F77FE
:103E00008E8747E016950795F794E7944A95D1F782
:103E10008E2D877089298F87AE01465F5F4F6BE0DB
:103E20008FEF0E94DC1DF9C00E949D1B7B018C015D
:103E3000DC01CB018F779070A070B070F601248107
:103E400033274427552782179307A407B50709F09E
:103E50000EC1D801C70180789F73A070B07037E0A1
:103E6000B695A795979587953A95D1F725813327EC
:103E70004427552782179307A407B50709F0F7C011
:103E8000D801C7018070907CAF71B0702EE0B695FC
:103E9000A795979587952A95D1F7268133274427AB
:103EA000552782179307A407B50709F0E0C080E003
:103EB00090E0A0EEB0E0E822F9220A231B2375E18E
:103EC00016950795F794E7947A95D1F72781822F75
:103ED0009927AA27BB2787709070A070B070E8164A
:103EE000F9060A071B0709F0C2C0922E9694969411
:103EF00096948281A82FBB27838199279695982F26
:103F0000882797958795A82BB92B109709F4AFC0F0
:103F1000092D112700FF09C0C5014696AC0160E0DC
:103F200070E0CD010E945621DC01109729F0BD01FF
:103F300080912F010E940C1CD5018D919C91892BA1
:103F400009F495C001FF93C0F50180898160808BE1
:103F50008EC0F6018281282F332783819927969579
:103F6000982F882797958795282B392B30933903DD
:103F70002093380352C0F6018281282F3327838192
:103F800099279695982F882797958795282B392BD1
:103F900030933C0320933B038481809349038581C4
:103FA00080933D03868180933E0380913A03816034
:103FB0001CC0F6013296AFE3B3E094E081918D939B
:103FC000915097FFFBCF80913A0382600EC0D601DB
:103FD0001296EFE3F3E093E08D9185839150319653
:103FE00097FFFACF80913A03846080933A0315C01B
:103FF00081E08093B50111C00E94781CF601828196
:104000000E94D80D0AC0F6018281882321F00E9407
:10401000951BFC0184810E94B10BD6018C919927DC
:104020008F77907020912F0133278217930749F4DF
:1040300080913703882329F0809137038150809342
:104040003703F50180899927969587959C01217002
:10405000307080FD04C0A90160E0C90106C0F5010F
:10406000468157816289808191810E94A61CCE0180
:1040700001960E94C306892B09F0C8CD2F960FB672
:10408000F894DEBF0FBECDBFDF91CF911F910F918E
:10409000FF90EF90DF90CF90BF90AF909F900895EA
:1040A000CF93DF93CDB7DEB726970FB6F894DEBF78
:1040B0000FBECDBF36E0FE01319611923A95E9F779
:1040C0004983AE014F5F5F4F0E94DC1D26960FB6FD
:1040D000F894DEBF0FBECDBFDF91CF910895CF938F
:1040E000DF93CDB7DEB726970FB6F894DEBF0FBECD
:1040F000CDBF26E0FE01319611922A95E9F7282FCF
:104100002F772983880F892F881F990B91958F7797
:104110008A83AE014F5F5F4F63E18FEF0E94DC1D2A
:1041200026960FB6F894DEBF0FBECDBFDF91CF91BC
:1041300008959F92AF92BF92CF92DF92EF92FF923B
:104140000F931F93CF93DF93CDB7DEB726970FB6AC
:10415000F894DEBF0FBECDBFFC018B01942E690128
:10416000672B11F0232B19F480E090E085C086E0E6
:104170005E010894A11CB11CD5011D928A95E9F736
:1041800054E1E52E8E2F8F778983EE0FEF2FEE1FF0
:10419000FF0BF1958E2F8F778A8320E08E2D992744
:1041A0008631910501F18731910534F4843191050F
:1041B00049F04597C9F024C08731910599F0489797
:1041C00081F01EC0802F8F778B83C801880F892FC5
:1041D000881F990B91958F778C83892D8F778D838D
:1041E0000FC023E02D5F2D5F92E0D5011296F601FE
:1041F000E20FF11D80818D9391502F5F97FFF7CFD4
:104200001092390310923803FF2480913803909163
:104210003903892B09F5AE014F5F5F4F6E2D8FEF8C
:104220000E94DC1D85E08093370306C08091370330
:10423000882341F00E9471048091380390913903E2
:10424000892BA1F3F3948091380390913903892B42
:1042500019F489E08F15F8F68091380390913903AD
:10426000009751F0E0913803F0913903E39488E12D
:104270008E1508F087CFCF0126960FB6F894DEBFD3
:104280000FBECDBFDF91CF911F910F91FF90EF90A7
:10429000DF90CF90BF90AF909F9008959A01462FE6
:1042A000BC0180E090E00E9499200895DF92EF9297
:1042B000FF920F931F93CF93DF93CDB7DEB726976F
:1042C0000FB6F894DEBF0FBECDBF9C017B018A0103
:1042D00001978F5F934008F050C086E0FE01319651
:1042E00011928A95E9F7822F8F778983220F232FE6
:1042F000221F330B3195822F8F778A8310923A03D6
:10430000DD2480913A03873031F1AE014F5F5F4F7A
:1043100060E18FEF0E94DC1D8FE08093370306C0C1
:1043200080913703882331F00E94710480913A0311
:104330008730B1F780913A03873029F082B7992707
:1043400088960E94DD08D39480913A03873019F053
:1043500089E08D15D0F680913A03873021F4809161
:104360003D038F3769F4E114F10411F0F701108275
:104370000115110511F0F801108280E090E018C0DD
:10438000E114F10421F080914903F70180830115C4
:10439000110551F08BE0F801ADE3B3E00D9001920F
:1043A0008A95E1F7F801138680913B0390913C03D5
:1043B00026960FB6F894DEBF0FBECDBFDF91CF912A
:1043C0001F910F91FF90EF90DF9008950F931F932F
:1043D000CF93DF93CDB7DEB726970FB6F894DEBF45
:1043E0000FBECDBF062F26E0FE01319611922A9511
:1043F000E9F7282F2F772983880F892F881F990B9A
:1044000091958F778A838FEF9FEF909339038093F5
:10441000380310E0809138039091390397FF20C052
:10442000AE014F5F5F4F602F8FEF0E94DC1D85E074
:104430008093370306C080913703882341F00E94A0
:10444000710480913803909139039923A4F31F5F7D
:10445000809138039091390397FF02C01A3000F31E
:10446000809138039091390326960FB6F894DEBFF9
:104470000FBECDBFDF91CF911F910F91089561E1E4
:104480000E94E621089562E10E94E6210895E199E3
:10449000FECF9FBB8EBBE09A99278DB3089541153F
:1044A000510569F0DC01E199FECF7FBB6EBBE09A5C
:1044B0006F5F7F4F0DB20D9241505040B1F708959C
:1044C000E199FECF9FBB8EBB6DBB0FB6F894E29A0D
:1044D000E19A0FBE0895DC0101C06D934150504038
:1044E000E0F70895FB01DC0101900D920020E1F757
:1044F00008950F931F93CF93DF93CDB7DEB72C971B
:104500000FB6F894DEBF0FBECDBF8C0136E03C8302
:1045100089839A832FEF3FE72D833E83CE01019657
:104520000E94CB22AF81B885A00FB11F1C922C96A0
:104530000FB6F894DEBF0FBECDBFDF91CF911F91B4
:104540000F9108950F931F93CF93DF93CDB7DEB7ED
:104550002C970FB6F894DEBF0FBECDBF8C013EE0A6
:104560003C8389839A832FEF3FE72D833E83CE01DF
:1045700001960E94CB22AF81B885A00FB11F1C927B
:104580002C960FB6F894DEBF0FBECDBFDF91CF9152
:104590001F910F9108952F923F924F925F926F92C9
:1045A0007F928F929F92AF92BF92CF92DF92EF92C3
:1045B000FF920F931F93CF93DF93CDB7DEB7629730
:1045C0000FB6F894DEBF0FBECDBFAA24BB24650191
:1045D0004C016D877E874F87588B44245524FC01FE
:1045E00046825782838181FD5BC28FEF9FEF6FC24E
:1045F00040FE44C2862D80538A30E0F4F0E36F160B
:1046000041F42A89222329F4772019F480E091E0EB
:104610008BC08AE09A89989F902D1124892F860D4E
:1046200080538A8B882314F4EFE7EA8B43FC38C26B
:104630007A8836C243FE05C0FA89FF2311F421E0CF
:104640002A8B862D992787FD90958836910554F5FC
:10465000853691050CF06BC08835910509F4D3C0FF
:1046600089359105B4F48B32910509F442C08C323E
:10467000910544F48032910509F43FC0839709F411
:1046800042C0F2C18D329105D9F18E9709F440C034
:10469000EBC18336910509F454C08436910509F4C1
:1046A00078C0E2C18037910509F4A5C08137910532
:1046B00084F48C369105B1F18D3691052CF4893650
:1046C000910509F466C0D0C18F36910509F490C0F8
:1046D000CBC18537910509F498C08637910524F43C
:1046E00083379105B9F1C0C18837910509F48BC0B2
:1046F000BBC180E190E0482A592AE0E2F0E005C021
:1047000080E890E011C0E0E4F0E04E2A5F2AC8C1E2
:1047100088E090E0482A592AEFEFFEEF4E225F2210
:104720001A8ABEC184E090E0482A592AB9C10F2EE6
:10473000FFE3AF2EF02D7A940F2EF3E66F2EF02DBF
:104740003AC1EF85F889CF0102968F87988BA080B8
:104750007A9431C1EF85F889CF0102968F87988BC3
:10476000A080B18043FE0BC0EA898E2F992787FD78
:104770009095BC01C5010E94B325898B07C0F50146
:1047800001900020E9F73197EA19E98BF9897F1A3E
:1047900012C142FE0BC0EF85F889CF0104968F87C6
:1047A000988B20813181428153810DC0EF85F8893A
:1047B000CF0102968F87988B808191819C0144273D
:1047C00037FD4095542F59016A01552364F4E2E006
:1047D000F0E04E2A5F2AD094C094B094A094A11C1B
:1047E000B11CC11CD11C8FEB9FEF482259222BC05A
:1047F00098E0998B0AC0E0E4F0E04E2A5F2A0F2E81
:10480000F8E76F2EF02DF0E1F98B42FE0BC0EF853B
:10481000F889CF0104968F87988B2081318142815E
:1048200053810BC0EF85F889CF0102968F87988B53
:10483000808191819C014427552759016A01EFEC41
:10484000FFEF4E225F221E010894211C311CF989C2
:10485000EF2EFF2400271127C601B501A8019701FB
:104860000E94CA25DC01CB01F10180838A301CF053
:10487000860D815203C0F1018081805DF101819339
:104880001F01C601B501A80197010E94CA2559015F
:104890006A012115310541055105F1F6CE01019658
:1048A000A22CA81AC20182739070892B09F07A9405
:1048B00046FE0FC0872D992787FD9095F989F03125
:1048C00031F40F2EFEEF7F2EF02D780E02C0782EE1
:1048D0007A9443FE12C08A89282F332727FD30950A
:1048E0008A2D9927821793072CF0E7EFFFEF4E22CE
:1048F0005F2203C0FA89FA19FA8B43FE03C02A89A2
:10490000721A01C07A18C20180789170892B69F4FB
:10491000872D7A9418164CF4B40180E290E00E943E
:104920008025872D7A941816BCF341FE04C0B4018B
:104930008DE290E00BC044FE04C0B4018BE290E035
:1049400005C045FE05C0B40180E290E00E948025CC
:1049500046FE0FC0B40180E390E00E948025898963
:10496000803139F4862D992787FD9095B4010E94F6
:10497000802550FE0DC0872D7A9418164CF4B40192
:1049800080E390E00E948025872D7A941816BCF36E
:1049900043FE11C08A89982F91509A8B18165CF4A7
:1049A000B40180E390E00E9480258A89E82FE150DD
:1049B000EA8B1816ACF3842D807869F4872D7A94ED
:1049C00018164CF4B40180E290E00E948025872DF7
:1049D0007A941816BCF3F3E66F1641F48A2D9927E2
:1049E00087FD9095B4010E9480252DC023E76216B3
:1049F000B1F489898150898B8F3F29F1F50180813C
:104A0000992787FD90950894A11CB11CB4010E94C0
:104A1000802599899150998B9F3F81F714C0CE01D1
:104A200001962816390679F08E010F5F1F4FF101AC
:104A300082911F01992787FD9095B4010E948025DE
:104A400020163106A1F7842D8078A9F0872D7A945D
:104A500018168CF4B40180E290E00E948025872D26
:104A60007A941816BCF307C0862D992787FD909578
:104A7000B4010E9480254424552412C0F5E26F162B
:104A800041F44424552443941A8A7A882AE0298BD5
:104A900007C0862D992787FD9095B4010E94802537
:104AA000F401838183FF08C0ED85FE85CF01019667
:104AB0008D879E87649005C0ED85FE856190ED87AA
:104AC000FE87662009F094CDF40186819781629675
:104AD0000FB6F894DEBF0FBECDBFDF91CF911F910F
:104AE0000F91FF90EF90DF90CF90BF90AF909F908D
:104AF0008F907F906F905F904F903F902F90089590
:104B00000F931F93CF93DF938C01EB018B81992738
:104B100081FF22C082FF14C02E813F814C815D81C4
:104B2000241735073CF4A881B9810D93A883B98374
:104B30002E813F812F5F3F4F2E833F83C8010EC0E0
:104B4000E885F985802F0995892B31F4EE81FF8165
:104B50003196EE83FF83F2CF8FEF9FEFDF91CF91FE
:104B60001F910F910895FC01615070400190011058
:104B7000D8F7809590958E0F9F1F0895991B79E027
:104B800004C0991F961708F0961B881F7A95C9F7DD
:104B900080950895A1E21A2EAA1BBB1BFD010DC032
:104BA000AA1FBB1FEE1FFF1FA217B307E407F507DD
:104BB00020F0A21BB30BE40BF50B661F771F881FB9
:104BC000991F1A9469F760957095809590959B014F
:084BD000AC01BD01CF01089505
:104BD800FFFF00010000FF0000F716FF0000951618
:104BE800FF0000F512FF00003B13FF01004715FF0F
:104BF80001004D13FF01007014FF01004416FFFF70
:00000001FF
